:020000040000FA
:040000007EEF0DF092
:08000800056ED8CF06F0E950A7
:10001000076EEA50086EE150096EE2500A6ED95040
:100020000B6EDA500C6EF350146EF450156EE050F7
:100030000D6E000100500F6E0150106E0250116ED7
:100040000350126E0450136E9DA22AEF00F09EB270
:100050001AEF0AF09DAA30EF00F09EBA91EF09F076
:100060000F50006E1050016E1150026E1250036E50
:100070001350046E0D50E06E0D8E0750E96E08505F
:10008000EA6E0950E16E0A50E26E0B50D96E0C50C8
:10009000DA6E1450F36E1550F46E055006C0D8FF9A
:1000A0001000F2CF0EF0F29EF76ABC0FF66E000E53
:1000B000F7220900F5500EBEF28E12000001020375
:1000C0000408090AF2CF0EF0F29EF76ADE0FF66E10
:1000D000000EF7220900F5500EBEF28E1200070640
:1000E000050403020100F76AF60FF66E000EF72210
:1000F0000900F55012000D0A43757272656E742086
:1001000073616D706C696E672064656C61792069DC
:100110007320256C64206D696C6C697365636F6E08
:1001200064732E0D0A00F76A360FF66E010EF72281
:100130000900F5501200456E7465722073616D7090
:100140006C696E672064656C617920696E206D69E9
:100150006C6C697365636F6E64733A200000F76AB4
:100160006E0FF66E010EF7220900F55012000D0A0F
:1001700053656C6563742061206368616E6E656CA5
:100180003A00F76A920FF66E010EF7220900F55059
:1001900012004368616E6E656C2025642074726184
:1001A0006E736D697420656E61626C65642C2049A4
:1001B00044206973203078254C782C20687973743A
:1001C0006572657369732069732025640D0A0000E8
:1001D000F76AE00FF66E010EF7220900F5501200E3
:1001E0004368616E6E656C202564207472616E7365
:1001F0006D69742064697361626C65642E0D0A0018
:10020000F76A100FF66E020EF7220900F550120081
:100210000D0A496E76616C6964206368616E6E6573
:100220006C2E2054727920616761696E2E00F76A26
:100230003E0FF66E020EF7220900F55012000D0A6D
:10024000456E74657220646573697265642043410C
:100250004E2069642E20546F2064697361626C655E
:100260002061206368616E6E656C2066726F6D2020
:100270000000F76A820FF66E020EF7220900F550B1
:1002800012007472616E736D697474696E672043D5
:10029000414E206D657373616765207365742069D5
:1002A000747320494420746F20626520302E000052
:1002B000F76AC00FF66E020EF7220900F550120021
:1002C0000D0A546865726520697320616C726561FE
:1002D00064792061206368616E6E656C2077697453
:1002E0006820746861742049443B207472792061ED
:1002F0006761696E210D0A00F76A080FF66E030E3A
:10030000F7220900F55012000D0A4368616E6E6510
:100310006C202564204944206973203078254C786E
:100320000D0A0000F76A340FF66E030EF72209007B
:10033000F550120053656E64207768656E2063681F
:10034000616E6765206265747765656E20726561B0
:1003500064696E67732069733A00F76A6A0FF66E14
:10036000030EF7220900F55012000D0A4879737444
:1003700065726573697320666F72206368616E6E63
:10038000656C2025642069732025640D0A00F76AD6
:100390009E0FF66E030EF7220900F55012000D0AAB
:1003A000232077726974696E6720636F6E66696770
:1003B00075726174696F6E20746F20656570726FFD
:1003C0006D00F2CF0EF0F29EF76ADC0FF66E030EB0
:1003D000F7220900F5500EBEF28E1200232072653E
:1003E0006164696E6720636F6E66696775726174B8
:1003F000696F6E2066726F6D20656570726F6D003B
:10040000F2CF0EF0F29EF76A1A0FF66E040EF72284
:100410000900F5500EBEF28E1200232073656E6443
:100420002064656C61793A20256C750D0A00F2CF65
:100430000EF0F29EF76A480FF66E040EF7220900DE
:10044000F5500EBEF28E120023206164635F63617B
:100450006E5F69645B25645D3D3078254C780D0ADC
:100460000000F2CF0EF0F29EF76A7C0FF66E040EDB
:10047000F7220900F5500EBEF28E120023206164AF
:10048000635F63616E5F68797374657265736973C6
:100490005B25645D3D25640D0A00F76AAA0FF66EC0
:1004A000040EF7220900F55012002320656E7465D2
:1004B00072696E6720636F6E6669677572617469D1
:1004C0006F6E206D6F646500F76AD80FF66E040ECC
:1004D000F7220900F550120031292053657420736A
:1004E000616D706C696E672064656C617900F76A94
:1004F000FE0FF66E040EF7220900F55012003229A5
:1005000020536574206368616E6E656C2070617243
:10051000616D65746572732028746F2073616D70EE
:100520006C652C2043414E2049442900F76A3C0F5A
:10053000F66E050EF7220900F5501200332920440B
:100540006F6E6500F76A540FF66E050EF72209000C
:10055000F55012000000F2CF0EF0F29EF76A700F15
:10056000F66E050EF7220900F5500EBEF28E12004F
:10057000232063616E6164632073746172747570AB
:100580000000F2CF0EF0F29EF76A9C0FF66E050E99
:10059000F7220900F5500EBEF28E12002320666984
:1005A000726D7761726520636F6D70696C65642030
:1005B00025730D0A0000F2CF0EF0F29EF76AD00FFD
:1005C000F66E050EF7220900F5500EBEF28E1200EF
:1005D00033302D4175672D303500F2CF0EF0F29E8D
:1005E000F76AF40FF66E050EF7220900F5500EBEFD
:1005F000F28E12002320707265737320616E792071
:100600006B657920696E20746865206E657874204A
:1006100074776F207365636F6E647320746F2065E9
:100620006E74657220636F6E666967206D6F6465B6
:100630000000F2CF0EF0F29EF76A4C0FF66E060E37
:10064000F7220900F5500EBEF28E12002320696ECB
:10065000697469616C697A696E672043414E2063F1
:100660006F6E74726F6C6C657200F2CF0EF0F29E5A
:10067000F76A840FF66E060EF7220900F5500EBEDB
:10068000F28E120023207374617274696E67206C9D
:100690006F6F70008C078D6B9EAAFED7AECF8EF069
:1006A0008E51080810E18D530DE08D078E519EA8E4
:1006B000FED7AD6E200E9EA8FED7AD6E8E519EA8C1
:1006C000FED7AD6E17D08E511F0814E28E517E08F2
:1006D00011E38C518D5D0EE28D518D2B036A8A25BD
:1006E000E96E8B510320EA6E8EC0EFFF8E519EA8FB
:1006F000FED7AD6E8E510D08CFE1036A8D518A256C
:10070000E96E8B510320EA6EEF6A000C006A016A01
:100710009151D89092B100260032013292B3002656
:100720000032013292B500260032013292B7002623
:100730000032013292B900260032013292BB00260B
:100740000032013292BD00260032013292BF0026F3
:100750000032013218EF04F08F6B8D6B0A0E8E6F32
:100760008C6B8A518B1103E1000E016EC1D08F5149
:100770008F2B036A8A25E96E8B510320EA6EEFCF37
:1007800090F090512D080DE1010E8D6F8F518F2B40
:10079000036A8A25E96E8B510320EA6EEFCF90F051
:1007A0000DD090512B080AE18F518F2B036A8A25B7
:1007B000E96E8B510320EA6EEFCF90F090512F0835
:1007C000D8B08ED090513908D8A08AD09051300836
:1007D00021E1036A8F518A25E96E8B510320EA6E6D
:1007E000EF5078080AE0036A8F518A25E96E8B5131
:1007F0000320EA6EEF5058080DE1100E8E6F8F2B1C
:100800008F518F2B036A8A25E96E8B510320EA6E84
:10081000EFCF90F08E510A081BE190512F0817E29C
:100820009051390814E30A0E916F8CC092F06ED784
:10083000300E905D01248C6F8F518F2B036A8A25B7
:10084000E96E8B510320EA6EEFCF90F0E6D748D0E7
:100850008E51100845E19051600806E290517A08E7
:1008600003E39051DF0B01D09051906F90512F080E
:1008700003E29051390806E29051400831E290516C
:1008800046082EE390512F080CE29051390809E3F5
:100890008C39916FF00E9117300E905D91258C6F11
:1008A00009D08C39916FF00E9117410E905D0A0FAF
:1008B00091258C6F8F518F2B036A8A25E96E8B519E
:1008C0000320EA6EEFCF90F09051600806E290515D
:1008D0007A0803E39051DF0B01D09051906FC6D797
:1008E0008D2D04D08E510A0801E18C6D8CC001F071
:1008F00084EF04F08B6B840E8A6F050E8C6FCADE5A
:100900008B6B840E8A6F28D701C089F089C001F0F3
:10091000000CEACF89F0E9CF88F082AF08D0888F49
:1009200088A9882B811F821F812BD8B4822B823902
:10093000F009846F8427E20F856F320F876F825131
:100940000F0B852785278727E90F866F8627862740
:1009500081390F0B8627872786378737871F873789
:1009600081510F0B87278437070E836F0A0E860786
:100970008727FDE385078627FDE384078527FDE3B9
:1009800083078427FDE3EA6A830EE96E070E881564
:10099000889DE906881507E188B9E92A88B903D056
:1009A000200E006E1CD0E926870EE95CD8B4888D35
:1009B000EF50006E08E188BD06D088B914D088B722
:1009C00002D0200E0BD088AF06D02D0E006EED5059
:1009D000889D889F04D088878899300E0026005013
:1009E0009EA8FED7AD6EEE5088ADDED7000C9151BB
:1009F0009303F3CF01F0F4CF00F09403F3500026FB
:100A000092519303F3500020026E78EF05F08F6B44
:100A10008D6B0A0E8E6F8C6B8B6B89518A1104E182
:100A2000000E016E026EE2D08F518F2B036A892572
:100A3000E96E8A510320EA6EEFCF90F090512D08B5
:100A40000DE1010E8D6F8F518F2B036A8925E96EA1
:100A50008A510320EA6EEFCF90F00DD090512B0811
:100A60000AE18F518F2B036A8925E96E8A51032091
:100A7000EA6EEFCF90F090512F08D8B0A9D09051E6
:100A80003908D8A0A5D09051300821E1036A8F51D0
:100A90008925E96E8A510320EA6EEF5078080AE052
:100AA000036A8F518925E96E8A510320EA6EEF505F
:100AB00058080DE1100E8E6F8F2B8F518F2B036A0C
:100AC0008925E96E8A510320EA6EEFCF90F08E51AE
:100AD0000A0821E190512F081DE2905139081AE3CC
:100AE000926B0A0E916F8CC094F08BC093F07FD7FD
:100AF000300E905D01248B6F000E02208C6F8F51A1
:100B00008F2B036A8925E96E8A510320EA6EEFCFA5
:100B100090F0E0D75DD08E5110085AE190516008F6
:100B200006E290517A0803E39051DF0B01D0905117
:100B3000906F90512F0803E29051390806E29051CE
:100B4000400846E29051460843E390512F0817E2CF
:100B50009051390814E38B35916F8C35926F913732
:100B600092379137923791379237F00E9117300EB6
:100B7000905D91258B6F000E92218C6F14D08B3578
:100B8000916F8C35926F91379237913792379137B9
:100B90009237F00E9117410E905D0A0F91258B6FE1
:100BA000000E92218C6F8F518F2B036A8925E96E7D
:100BB0008A510320EA6EEF50906F600806E2905170
:100BC0007A0803E39051DF0B01D09051906FB1D7B9
:100BD0008E510A0807E18D2D05D08B1F8C1F8B2BA2
:100BE000D8B48C2B8BC001F08CC002F002EF06F061
:100BF0008B6B800E8A6F070E8C6F4CDD8A6B800EBC
:100C0000896F05D702C088F001C087F087C001F066
:100C100088C002F042EF06F0806B805173EC00F068
:100C2000802B006E00509EA8FED7AD6E1C0E805D1E
:100C3000F4E1100EE96E5BC082F05AC081F069DE0B
:100C40001F0E816F815173EC00F0812B006E0050FC
:100C50009EA8FED7AD6E2F0E815DF4E1806B8051B2
:100C600093EC00F0000905E0802B9EA8FED7AD6E46
:100C7000F6D70D0E9EA8FED7AD6E0A0E9EA8FED723
:100C8000AD6EB6D702C07FF001C07EF07FC05BF0D2
:100C90007EC05AF003EF0AF09151016A905D03E2C1
:100CA00090C000F00CD0006A080E926F90370036AA
:100CB0009151005CD8B0006E0136922FF7D7000C2E
:100CC000200E8BA9300E8C6F8AC000F08AAF07D03F
:100CD000001E002A00C08AF02D0E8C6F8B8F0150F1
:100CE0008AC090F0640E916FD7DF00C08AF0300E9A
:100CF00001248D6F8AC090F00A0E916FCDDF300E07
:100D000000248F6F300E01248E6F8CC000F08BA7F3
:100D100002D08BAF8B958BB90BD08BAF22D08BB51C
:100D200020D000C08DF08BB31CD000C08EF019D045
:100D3000300E8D5D16E100C08DF0200E8C6F8BA7FC
:100D400004D08B958B838BAF8B93300E8E5D09E136
:100D500000C08EF0200E8D6F8BA7F7D78B938BAFD3
:100D60008B918BA504D08C519EA8FED7AD6E8BA322
:100D700004D08D519EA8FED7AD6E8BA104D08E51AC
:100D80009EA8FED7AD6E8F519EA8FED7AD6E000C0B
:100D90008ABF10D00F0E006E893900160A0E005C53
:100DA00003E2300E002602D08A51002600509EA891
:100DB000FED7AD6E0F0E89170A0E895D02E2300E66
:100DC00002D08A9F8A51892789519EA8FED7AD6E8D
:100DD000000C9EAAFED7AECF86F086519EA8FED705
:100DE000AD6E8651390805E3300E865D016E0FD079
:100DF0000ED08651600806E286517A0803E38651D8
:100E0000DF0B01D08651BF0F0A0F016E00D0000C1E
:100E1000E0DF01C085F0DDDF01C084F08451DD0832
:100E200004E185C001F007D006D08551100DF350C4
:100E30008425016E00D0000C846B8451AFEC00F06F
:100E4000000905E0842B9EA8FED7AD6EF6D70D0EE7
:100E50009EA8FED7AD6E0A0E9EA8FED7AD6E7E6B25
:100E60007E510708D8A08DD0D8907E35036A3E0FFA
:100E7000E96E000E0320EA6EECCF03F0ED52EF5066
:100E800002E103525CE0D8907E35036A3E0FE96EC2
:100E9000000E0320EA6EECCF85F0ED52EFCF84F028
:100EA000036A7E514E0FE96E000E0320EA6EEFCF0B
:100EB00086F0876B8751C1EC00F0872B006E0050E5
:100EC0009EA8FED7AD6E080E875DF4E17EC08AF065
:100ED0001F0E8B6FF5DE0A0E886F8851C1EC00F093
:100EE000882B006E00509EA8FED7AD6E250E885D43
:100EF000F4E185C089F0570E8A6F4ADF84C089F01B
:100F0000570E8A6F45DF280E896F8951C1EC00F0BA
:100F1000892B006E00509EA8FED7AD6E380E895DFD
:100F2000F4E186C08AF01F0E8B6FCADE0D0E9EA8FC
:100F3000FED7AD6E0A0E9EA8FED7AD6E20D0846B94
:100F40008451E8EC00F0842B006E00509EA8FED780
:100F5000AD6E080E845DF4E17EC08AF01F0E8B6FCB
:100F6000AFDE0A0E856F8551E8EC00F0852B006E30
:100F700000509EA8FED7AD6E1F0E855DF4E17E2B5E
:100F80006FD7B8DC01C07FF07F51070814E2846B93
:100F9000845100EC01F0000905E0842B9EA8FED7E7
:100FA000AD6EF6D70D0E9EA8FED7AD6E0A0E9EA8AA
:100FB000FED7AD6E41D7846B845117EC01F0000968
:100FC00005E0842B9EA8FED7AD6EF6D70D0E9EA829
:100FD000FED7AD6E0A0E9EA8FED7AD6E846B84510F
:100FE00039EC01F0000905E0842B9EA8FED7AD6E18
:100FF000F6D70D0E9EA8FED7AD6E0A0E9EA8FED7A0
:10100000AD6E06DF01C080F003DF01C081F080C05B
:1010100083F081C082F0825302E1835330E07F513C
:101020007E5D2DE07E6B7E51070829E3D8907E35EA
:10103000036A3E0FE96E000E0320EA6EECCF85F0E6
:10104000ED52EFCF84F08251845D17E18351855DCD
:1010500014E1846B845158EC01F0000905E0842B05
:101060009EA8FED7AD6EF6D70D0E9EA8FED7AD6E2C
:101070000A0E9EA8FED7AD6E9ED77E2BD4D7D890F1
:101080007F35036A3E0FE96E000E0320EA6E83C0CF
:10109000ECFFED5282C0EFFFD8907F35036A3E0F20
:1010A000E96E000E0320EA6EECCF85F0ED52EFCF33
:1010B00084F0866B86517CEC01F0862B006E00502C
:1010C0009EA8FED7AD6E0A0E865DF4E17FC08AF061
:1010D0001F0E8B6FF5DD0C0E876F87517CEC01F0D6
:1010E000872B006E00509EA8FED7AD6E150E875D53
:1010F000F4E185C089F0570E8A6F4ADE84C089F01A
:10110000570E8A6F45DE0D0E9EA8FED7AD6E0A0EF5
:101110009EA8FED7AD6E846B845192EC01F000095D
:1011200005E0842B9EA8FED7AD6EF6D70D0E9EA8C7
:10113000FED7AD6E0A0E9EA8FED7AD6E7AEC04F017
:1011400001C07EF0120E7F25846FA96E7EC0A8FFBD
:10115000A69CA69EA684F2CF00F0F29E0F01550E2B
:10116000A76EAA0EA76EA682A6B2FED7A6940050BE
:10117000F212036A00017F514E0FE96E000E032048
:10118000EA6E7EC0EFFF036A7F514E0FE96E000EDC
:101190000320EA6EEFCF84F0856B8551ADEC01F052
:1011A000852B006E00509EA8FED7AD6E190E855D92
:1011B000F4E17FC08AF01F0E8B6F82DD1B0E866FFD
:1011C0008651ADEC01F0862B006E00509EA8FED734
:1011D000AD6E1F0E865DF4E184C08AF01F0E8B6F2A
:1011E0006FDD0D0E9EA8FED7AD6E0A0E9EA8FED72F
:1011F000AD6E03EF0AF084C085F082C0A9FF84C001
:10120000A8FFA69CA69EA684F2CF00F0F29E0F0136
:10121000550EA76EAA0EA76EA682A6B2FED7A694FA
:101220000050F212010E00018225856F83C086F006
:10123000A96E83C0A8FFA69CA69EA684F2CF00F04C
:10124000F29E0F01550EA76EAA0EA76EA682A6B239
:10125000FED7A6940050F2120001000C806B805162
:10126000C7EC01F0000905E0802B9EA8FED7AD6E0B
:10127000F6D70D0E9EA8FED7AD6E0A0E9EA8FED71D
:10128000AD6E826B5BC084F05AC083F0B4DF7E6BBE
:10129000020E7F6F7E51070819E3D8907E35036AEE
:1012A0003E0FE96E000E0320EA6EECCF81F0ED52A6
:1012B000EFCF80F07FC082F081C084F080C083F0E7
:1012C0009ADF7E517E2B020E7F27E4D77E6B120EB3
:1012D0007F6F7E51070823E3036A7E514E0FE96E4C
:1012E000000E0320EA6EEFCF80F07FC0A9FF80C020
:1012F000A8FFA69CA69EA684F2CF00F0F29E0F0146
:10130000550EA76EAA0EA76EA682A6B2FED7A69409
:101310000050F21200017E517E2B7F2BDAD7EEEFC8
:1013200009F09EAAFED7AE509D9A7E6B7E514DEC81
:1013300002F0000905E07E2B9EA8FED7AD6EF6D721
:101340000D0E9EA8FED7AD6E0A0E9EA8FED7AD6EFE
:101350007E6B7E5164EC02F0000905E07E2B9EA8B6
:10136000FED7AD6EF6D70D0E9EA8FED7AD6E0A0E57
:101370009EA8FED7AD6E7E6B7E5177EC02F0000921
:1013800005E07E2B9EA8FED7AD6EF6D70D0E9EA86B
:10139000FED7AD6E0A0E9EA8FED7AD6E7E6B7E5157
:1013A00096EC02F0000905E07E2B9EA8FED7AD6EFC
:1013B000F6D70D0E9EA8FED7AD6E0A0E9EA8FED7DC
:1013C000AD6E7AEC04F00150010A05E0030A04E076
:1013D000010A03E017D020D42FD540D77E6B7E5171
:1013E000A2EC02F0000905E07E2B9EA8FED7AD6EB0
:1013F000F6D70D0E9EA8FED7AD6E0A0E9EA8FED79C
:10140000AD6E15D0A5D77E6B7E51A2EC02F000091F
:1014100005E07E2B9EA8FED7AD6EF6D70D0E9EA8DA
:10142000FED7AD6E0A0E9EA8FED7AD6E91D79E9ADE
:1014300030EF00F0562AD8B4572A582AD8B4592A7F
:101440005A50585C06E15B50595C03E15C80596A74
:10145000586A5650E70805E15750030802E1576AF9
:10146000566A9E9230EF00F0F2CF67F0F29E64C0B1
:10147000A9FFA69CA69EA680A85067BFF28E656FA6
:10148000010E6425F2CF68F0F29EA96EA69CA69E7E
:10149000A680A85068BFF28E666F65C003F066C074
:1014A00001F065C002F0000CEACF6BF0E9CF6AF002
:1014B0006439F009666F6627E20F676F320F696F54
:1014C00064510F0B672767276927E90F686F682743
:1014D000682763390F0B6827692768376937691FE1
:1014E000693763510F0B69276637070E656F0A0E60
:1014F00068076927FDE367076827FDE36607672735
:10150000FDE365076627FDE3EA6A650EE96E070EEF
:101510006A156A9DE926690EE95CD8B46A8DEF50B8
:10152000006E08E16ABD06D06AB90CD06AB702D075
:10153000200E03D06A876A99300E002600509EA8BC
:10154000FED7AD6EEE506AADE6D7D4EF0AF0626B0F
:101550006251E1EC01F0000905E0622B9EA8FED784
:10156000AD6EF6D70D0E9EA8FED7AD6E0A0E9EA8E4
:10157000FED7AD6E646B78DF02C05BF001C05AF03D
:10158000626B625100EC02F0622B006E00509EA86C
:10159000FED7AD6E0E0E625DF4E1100EE96E5BC01B
:1015A00064F05AC063F080D70D0E9EA8FED7AD6ED2
:1015B0000A0E9EA8FED7AD6E606B020E616F605181
:1015C000070870E3D8906035036A3E0F016E000E85
:1015D000032201C062F003C063F061C064F044DF25
:1015E00063C0EAFF62C0E9FF02C0ECFFED5201C038
:1015F000EFFFD8906035036A3E0FE96E000E0320BE
:10160000EA6EECCF63F0ED52EFCF62F0646B6451A1
:1016100017EC02F0642B006E00509EA8FED7AD6E52
:101620000D0E645DF4E1176AF2BE178EF29E60C083
:101630008AF01F0E8B6F60EC06F017BEF28E0F0E55
:10164000656F655117EC02F0652B006E00509EA887
:10165000FED7AD6E130E655DF4E1176AF2BE178E0C
:10166000F29E63C089F0570E8A6FC8EC06F017BE71
:10167000F28E176AF2BE178EF29E62C089F0570E84
:101680008A6FC8EC06F017BEF28E0D0E9EA8FED72C
:10169000AD6E0A0E9EA8FED7AD6E6051602B020E95
:1016A00061278DD7606B120E616F6051070855E39B
:1016B000036A60514E0FE96E000E0320EA6EF2CF0E
:1016C00064F0F29E61C0A9FFA69CA69EA680A850C9
:1016D00064BFF28EEF6E036A60514E0FE96E000E2A
:1016E0000320EA6EEFCF62F0636B635131EC02F0DE
:1016F000632B006E00509EA8FED7AD6E150E635D85
:10170000F4E1176AF2BE178EF29E60C08AF01F0ED7
:101710008B6F60EC06F017BEF28E5D0E9EA8FED7B2
:10172000AD6E3D0E9EA8FED7AD6E176AF2BE178E47
:10173000F29E62C08AF01F0E8B6F60EC06F017BE3F
:10174000F28E0D0E9EA8FED7AD6E0A0E9EA8FED795
:10175000AD6E6051602B612BA8D7CEEF0DF0C0505D
:10176000C00B0709C06EC08EC280C150C00BC16ED5
:10177000DBEF0DF0EA6A610EE96EEF500FE0050E47
:10178000016E006A002EFED7012EFBD72E0E006ED2
:10179000002EFED700000000EF2EF1D7F6EF0DF07F
:1017A0006039700B006ED89000361F0E6F14001059
:1017B0006F6E6ECF00F0003A0030070B605DF9E10C
:1017C000000C010E706EB80E716E050E726E85EF14
:1017D0000CF071C078F070C077F0765352E077C0AB
:1017E000E9FF78C0EAFF72C0EFFF7751D8B47807FD
:1017F000770777C0E9FF78C0EAFF73C0EFFF775142
:10180000D8B47807770777C0E9FF78C0EAFF74514A
:10181000030BEF6E77C0E9FF78C0EAFF74C000F0F9
:10182000003600360036F80E00160050E00BEF10C0
:10183000EF6E77C0E9FF78C0EAFFEF500809EF6E5E
:101840007751D8B47807770777C0E9FF78C0EAFF07
:1018500074C000F0003A0032070E00160050070B6B
:10186000EF6E77C0E9FF78C0EAFF75C000F0003680
:1018700000360036F80E00160050F80BEF10EF6E31
:101880003FD077C0E9FF78C0EAFFEF6A7751D8B45C
:101890007807770777C0E9FF78C0EAFFEF6A7751EA
:1018A000D8B47807770777C0E9FF78C0EAFF72C03D
:1018B00000F0003A0036E00E00160050E00BEF6E2C
:1018C0007751D8B47807770777C0E9FF78C0EAFF87
:1018D00072C000F00032003200321F0E00160050BD
:1018E0001F0BEF6E77C0E9FF78C0EAFF73C000F00E
:1018F000003A0036E00E00160050E00BEF10EF6EDD
:10190000000C040E606F4CDF5CD7606A9F0E6014A1
:10191000606E608460CF50FF739A73980F0E716F82
:101920001B0E706F756B746B736B726B010E766F41
:1019300050DF0F0E716F030E706F756B746B736BEE
:10194000726B010E766F45DF0F0E716F070E706FB1
:10195000756B746B736B726B010E766F3ADF0F0EE3
:10196000716F1F0E706F756B746B736B726B010E02
:10197000766F2FDF0F0E716F0B0E706F756B746BC0
:10198000736B726B010E766F24DF0F0E716F706FC9
:10199000756B746B736B726B010E766F1ADF0F0EC3
:1019A000716F130E706F756B746B736B726B010ECE
:1019B000766F0FDF0F0E716F170E706F756B746B94
:1019C000736B726B010E766F04DF9350FB0B08098B
:1019D000936E606BE5DE13EF0EF0606B60510708ED
:1019E00025E3036A605151EC00F0616F6135006ED0
:1019F0000036FC0E0016C250C30B0010C26E036A04
:101A0000605162EC00F0006ED89000360050036A1E
:101A10001E0FE96E000E0320EA6EC282C2B2FED72C
:101A2000C3CFEFFFC4CFECFF602BD8D727EF0EF06A
:101A30000F0E6E6F660E6D6F0F0140B708D0F10E7E
:101A40006F1408096F6E00016F6B1BD00F0130B768
:101A500009D0F10E6F1406096F6E010E00016F6F51
:101A600010D00F0120B709D0F10E6F1404096F6E6A
:101A7000020E00016F6F05D00F01000E016E3BD00A
:101A800000016951030B006EFC0E60140010606EC3
:101A90000F0E716F640E706F65C075F064C074F0E6
:101AA00063C073F062C072F06AC076F092DE68C004
:101AB00065FF659C6BB1658C6C6B68516C5D14E265
:101AC00066C0E9FF67C0EAFFEFCF72F06EC0EAFFC1
:101AD0006DC0E9FF72C0EFFF6D2BD8B46E2B662B83
:101AE000D8B4672B6C2BE9D76086F10E6F146F6E3C
:101AF000010E016E0F01000103EF0FF0F86AD09E96
:101B00000D8EEA6AE96AC150C00B0F09C16EB88632
:101B1000440EAF6E000EB06E260EAC6E900EAB6E25
:101B2000186A196A010E1A6E1B6A1C6A1D6A606BBC
:101B30006051ABEC02F0000905E0602B9EA8FED7D7
:101B4000AD6EF6D70D0E9EA8FED7AD6E0A0E9EA8FE
:101B5000FED7AD6E606B6051C1EC02F0602B006E81
:101B600000509EA8FED7AD6E140E605DF4E1616B6F
:101B70006151DBEC02F0000905E0612B9EA8FED765
:101B8000AD6EF6D70D0E9EA8FED7AD6E0A0E9EA8BE
:101B9000FED7AD6E576A566A5C90D9D45A5202E1AC
:101BA0005B5204E05A3C06D05B3C04D0010E5B6EF5
:101BB000F40E5A6ED4D5606B6051EDEC02F0000962
:101BC00005E0602B9EA8FED7AD6EF6D70D0E9EA841
:101BD000FED7AD6E0A0E9EA8FED7AD6E9D8AC00ED2
:101BE000F212080E606FFA0E616FC4D5602FFBD73A
:101BF0009D9A000E0509CA6EF90ECB6E9D82606B30
:101C0000605119EC03F0000905E0602B9EA8FED797
:101C1000AD6EF6D70D0E9EA8FED7AD6E0A0E9EA82D
:101C2000FED7AD6E6ED6606B605135EC03F00009E7
:101C300005E0602B9EA8FED7AD6EF6D70D0E9EA8D0
:101C4000FED7AD6E0A0E9EA8FED7AD6EC6D6000EAC
:101C50005CB0010E0108D8A4F8D05D6A5D50070899
:101C6000D8A0F2D05D50070820E0D8905D34036A18
:101C70001E0FE96E000E0320EA6EECCF61F0ED520C
:101C8000EFCF60F00A0EE96E176AF2BE178EF29E71
:101C900061C082F060C081F089EC04F017BEF28E62
:101CA0002C0E9EA8FED7AD6E23D0D8905D34036A6B
:101CB0001E0FE96E000E0320EA6EECCF61F0ED52CC
:101CC000EFCF60F00A0EE96E176AF2BE178EF29E31
:101CD00061C082F060C081F089EC04F017BEF28E22
:101CE0000D0E9EA8FED7AD6E0A0E9EA8FED7AD6E55
:101CF000D8905D34036A3E0FE96E000E0320EA6E51
:101D0000ECCF03F0ED52EF5003E10352D8B47BD097
:101D1000D8905D34036A2E0FE96E000E0320EA6E40
:101D2000ECCF61F0ED52EFCF60F0D8905D34036AF4
:101D30001E0FE96E000E0320EA6EECCF03F0ED52A9
:101D4000EF50605D626F03506159636F036E6251C3
:101D500063AF08D0000ED8806255006E000E635548
:101D6000036E0050636F03C064F0036A5D504E0F52
:101D7000E96E000E0320EA6EEF5000AE03D064AFB0
:101D800008D002D064BF3FD0645303E1635D3BE001
:101D90003AE3D8905D34036A1E0FE96E000E03200B
:101DA000EA6EECCF61F0ED52EFCF60F0D8905D3489
:101DB000036A1E0FE96E000E0320EA6EECCF64F09A
:101DC000ED52EFCF63F060C05FF064C05EF0D8907A
:101DD0005D34036A3E0FE96E000E0320EA6EECCF1D
:101DE00061F0ED52EFCF60F0656B646B61C063F042
:101DF00060C062F0676B5E0E666F020E686F696BA3
:101E00006A6B6B6B15D6D8905D34036A2E0F016E2A
:101E1000000E032203C061F0D8905D34036A1E0FE8
:101E2000E96E000E0320EA6EECCF03F0ED52EFCF27
:101E300062F061C0EAFF01C0E9FF03C0ECFFED52B0
:101E400062C0EFFF5D2A0AD75C9000D70000030054
:0200000400F00A
:1000000000FA1234000000000000000000000000B0
:1000100000000A00000000000000000000000000D6
:020020000000DE
:020000040030CA
:0E00000000061E1E008281000FC00FE00F40A0
:00000001FF
